:020000040000FA
:10000000F428B400841780048413A201201CA200E9
:1000100023200319EF2823200319EF282320EF289A
:10002000B4007120200821040319EF28E92084136B
:100030003408800664001C281D28A00A0319A10F9B
:100040001A288006EF283408A2060130A000A1017A
:10005000000834052206031D0800A00A0319A10F99
:1000600028280800A600360884000930A7000310DD
:100070003E20A60CA70B382803143E288413B31D7A
:100080004D2800083404331D34068000841700080E
:100090003404031C34068000582800083404031C70
:1000A0003406331934068000841734098005582833
:1000B00000308A00330D0639A0006520A100003011
:1000C0008A00200A652000008328693E03188A0AF6
:1000D00082000134713403341134003438340C3468
:1000E000D534FF3A84178005EF28A301A200FF3022
:1000F000A207031CA307031CEF280330A100DF3075
:1001000083207728A101E83EA000A109FC30031C50
:100110008C28A00703188928A0076400A10F89284C
:1001200020189228A01C9628000096280800A200FB
:100130000330A328A2000130A328A2000630A32880
:10014000A2000430A328A80023082102031DAA2826
:100150002208200204300318013003190230280558
:10016000031DFF30EF280404031DFF30EF28A50115
:10017000A4011030A600210DA40DA50D2208A40293
:100180002308031C230FA5020318CD282208A40767
:1001900023080318230FA5070310A00DA10DA60B1C
:1001A000BB282008EF281030A800A101A001A70C4F
:1001B000A60C031CE1282208A00723080318230F1C
:1001C000A107A10CA00CA50CA40CA80BD7282408EF
:1001D000EF28A009A109A00A0319A10A08008313A6
:1001E000031383126400080088308B008316673085
:1001F0008F00831207309900850183160A3085002D
:1002000052309F00831285309F0005168316051219
:100210008312051583160511831205108316051028
:1002200083126D30BE000130BF006830C000013065
:10023000C1004B102030850683168512831252228E
:100240004208BA004308BB006400851D1A296400F7
:10025000851927290130A0000530840008300120CD
:100260002008BC002108BD003C08A0003D08A100FA
:10027000A3010530A020031D1A293C08A0003D0859
:10028000A100A3010F309720031D72293A08B8007E
:100290003B08B9003A08A0003B08A1000130A300C8
:1002A000AE309A20C6003A08A0003B08A100A30186
:1002B000AF30A020C800460884004808B320C8001A
:1002C000C90064004808490403196829BA016E2965
:1002D000AF30BA020030031C013EBB020A30BC0042
:1002E000BD01A22A3C08A0003D08A100A3011930CD
:1002F0009720031D852905108316051083121430DD
:10030000BC00BD010230BA00A22A3C08A0003D0892
:10031000A100A30123309720031DA2293808A000C3
:100320003908A1003F08A3003E089D20031D9C2919
:1003300005148316051083121E30BC00BD01033066
:10034000BA00A22A3C08A0003D08A100A3012D305C
:100350009720031DB429BE0A0319BF0A2830BC0028
:10036000BD010430BA00A22A3C08A0003D08A1004B
:10037000A30137309720031DC9290130BE02003088
:10038000031C013EBF023230BC00BD010530BA0083
:10039000A22A3C08A0003D08A100A30141309720FB
:1003A000031DDB29C00A0319C10A3C30BC00BD0192
:1003B0000630BA00A22A3C08A0003D08A100A30113
:1003C0004B309720031DF0290130C0020030031C80
:1003D000013EC1024630BC00BD010730BA00A22A6E
:1003E0003C08A0003D08A100A30155309720031D43
:1003F000072A6D30BE000130BF006830C0000130F8
:10040000C1005030BC00BD010830BA00A22A3C082F
:10041000A0003D08A100A3015F309720031D222A00
:1004200005148316051083120130A300F4307620E2
:1004300005108316051083125A30BC00BD01093027
:10044000BA00A22A3C08A0003D08A100A30169301F
:100450009720031D322A4B106430BC00BD010A30C6
:10046000BA00A22A3C08A0003D08A100A3017330F5
:100470009720031D422A4B146E30BC00BD010B3087
:10048000BA00A22A3C08A0003D08A100A3017D30CB
:100490009720031D512A7830BC00BD010130BA00FD
:1004A000A22A1A29BA01BB010130CA0064006530D2
:1004B0004A020318712A9F1464009F1C602A5C2A58
:1004C0001E08C50083161E088312C4004408BA071C
:1004D00045080318013EBB0764008519A12ACA0F0D
:1004E000562A3A08A0003B08A1006430A200A301EC
:1004F000B720BA002108BB00E030A000F630A10010
:100500003A08A2003B08A300B720BA002108BB00AC
:100510003A08A6003B08A7000230A200A301D3209E
:10052000C2002508C3004208A0004308A100013012
:10053000A3002C309720031DA12A05108316051057
:1005400083120800051283160512023083127520EB
:10055000051683160512640083124B18B82A05305D
:10056000B6000430B4000230B3003A083220BF2A8B
:100570000530B6000430B400B3013A0832203C081C
:10058000A0003D08A10005308400103010201A2979
:10059000FF3FFF3FFF3FFF3FFF3FFF3FFF3FFF3F6B
:1005A000FF3FFF3FFF3FFF3FFF3FFF3FFF3FFF3F5B
:1005B000FF3FFF3FFF3FFF3FFF3FFF3FFF3FFF3F4B
:1005C000FF3FFF3FFF3FFF3FFF3FFF3FFF3FFF3F3B
:02400E00DC3C98
:08400000FF3FFF3FFF3FFF3FC0
:00000001FF
